:100000004AC100000C94E6080C94BB080C949008BC
:100010000C9465080C943A080C940F086DC100000C
:100020006BC1000069C1000067C1000065C100002C
:1000300063C1000061C100005FC100005DC100003C
:100040005BC1000059C1000057C1000055C100004C
:1000500053C1000051C100004FC1000096C700000D
:100060004BC100005CC7000031C7000045C1000063
:1000700043C1000041C100003FC100003DC100007C
:100080003BC1000039C1000037C1000035C100008C
:1000900033C1000031C100002FC100002DC100009C
:1000A0002BC1000029C1000027C1000025C10000AC
:1000B00023C1000021C100001FC100001DC10000BC
:1000C0001BC1000019C1000017C1000015C10000CC
:1000D00013C1000011C100000FC100000DC10000DC
:1000E0000BC100002F0A002300230023005C232300
:1000F00023235265616C53696D476561722300006B
:10010000002100240027002A002D003000330001C8
:10011000010000040107010A010000220025002857
:10012000002B002E00310034000201000005010800
:10013000010B01000020002300260029002C002FC5
:100140000032000001000003010601090105050558
:1001500005070508080808020202020A0A0808043E
:10016000040404010101010101010103030303036C
:10017000030303040707070C0C0C0C0C0C0C0C02FB
:1001800002020206060606060606060B0B0B0B0B02
:100190000B0B0B01021020200808102040102040FB
:1001A000800201020108040201010204081020403B
:1001B0008080402010080402018004020180402059
:1001C0001008040201080402010102040810204082
:1001D00080010204081020408000000A0B02090C74
:1001E0000D0E0807030401000000000000000000DD
:1001F00000000000000000000000000000000000FF
:1002000000000000001211100000000000000000BB
:100210000000000000000000000000000000002FAF
:100220000A002300230023005C232323235265615B
:100230006C53696D4765617223003D300A003D31A2
:100240000A000A003D300A003D310A0042544E5F68
:10025000444952454354323D300A003D300A004281
:10026000544E5F444952454354323D310A003D31BA
:100270000A000A000A002F0A002300230023005C62
:10028000232323235265616C53696D476561722393
:1002900000001109F80E11241FBECFEFD1E2DEBF1E
:1002A000CDBF00E00CBF2BE0ACE5B6E001C01D9275
:1002B000AB34B207E1F716E0A0E0B2E0E6E3F3E228
:1002C00000E00BBF02C007900D92AC35B107D9F723
:1002D00011E0CAE4D1E000E006C021970109802FB7
:1002E000FE010E94650FC934D10780E00807A9F715
:1002F0000E94220A0C948A1183CEAF92BF92CF92B1
:10030000DF92EF92FF920F931F93CF93DF936C01D5
:100310007B018B01040F151FEB015E01AE18BF08B6
:10032000C017D10759F06991D601ED91FC91019068
:10033000F081E02DC6011995892B79F7C501DF9170
:10034000CF911F910F91FF90EF90DF90CF90BF90D2
:10035000AF900895EFEAF7E04481558160817181A3
:1003600083E097E0CACFFC01538D448D252F30E008
:10037000842F90E0821B930B541710F0CF960895B2
:1003800001970895FC01918D828D981761F0A28DDF
:10039000AE0FBF2FB11D5D968C91928D9F5F9F73A5
:1003A000928F90E008958FEF9FEF0895FC01918D5B
:1003B000828D981731F0828DE80FF11D858D90E0C8
:1003C00008958FEF9FEF0895FC01918D228D892F65
:1003D00090E0805C9F4F821B91098F73992708954D
:1003E00083E097E0F1DF21E0892B09F420E0822F00
:1003F0000895FC01A48DA80FB92FB11DA35ABF4FBA
:100400002C91848D90E001968F739927848FA68913
:10041000B7892C93A089B1898C91837080648C9367
:10042000938D848D981306C00288F389E02D808116
:100430008F7D80830895EF92FF920F931F93CF9348
:10044000DF93EC0181E0888F9B8D8C8D98131AC00F
:10045000E889F989808185FF15C09FB7F894EE89F6
:10046000FF896083E889F989808183708064808353
:100470009FBF81E090E0DF91CF911F910F91FF909E
:10048000EF900895F62E0B8D10E00F5F1F4F0F7346
:100490001127E02E8C8D8E110BC00FB607FCFACF02
:1004A000E889F989808185FFF5CFCE01A2DFF2CFFF
:1004B000EB8DEC0FFD2FF11DE35AFF4FF0829FB73C
:1004C000F8940B8FEA89FB8980818062D0CF0F93EB
:1004D0001F93CF93DF938C01D0E0C0E0F801EC0FC5
:1004E000FD1F6491662339F083E097E0A4DF892B38
:1004F00011F02196F3CFCE01DF91CF911F910F9193
:100500000895CF93DF93EC01888D8823B1F0AA89F9
:10051000BB89E889F9898C9185FD03C0808186FDBE
:100520000CC00FB607FCF7CF8C9185FFF2CF80810E
:1005300085FFEDCFCE015DDFEACFDF91CF9108954A
:100540008150823108F05AC0E82FF0E08827E45546
:10055000FD4F8F4F0C94650FCC02D002BE02C40237
:10056000C802FE02D302D902DD02E302E702EB0277
:10057000F102F502FE02F902FF02030380918000FE
:100580008F77809380000895809180008F7DF9CFD0
:1005900080918000877FF5CF84B58F7784BD0895E3
:1005A00084B58F7DFBCF8091B0008F778093B000B2
:1005B00008958091B0008F7DF9CF809190008F7762
:1005C000809390000895809190008F7DF9CF809165
:1005D0009000877FF5CF8091A0008F778093A00057
:1005E00008958091A0008F7DF9CF8091A000877F32
:1005F000F5CF809120018F7780932001089580911D
:1006000020018F7DF9CF80912001877FF5CFCF9397
:10061000DF93282F30E0F901E752FE4F8491F90172
:10062000ED56FE4FD491F901E35BFE4FC491CC230C
:1006300099F0811185DFEC2FF0E0EE0FFF1FED5CEC
:10064000FE4FA591B491EC91ED2381E090E009F487
:1006500080E0DF91CF91089580E090E0FACF1F9382
:10066000CF93DF93282F30E0F901E752FE4F8491BA
:10067000F901ED56FE4FD491F901E35BFE4FC491B1
:10068000CC23A1F0162F81115BDFEC2FF0E0EE0FF1
:10069000FF1FE75EFE4FA591B4918FB7F894EC91E0
:1006A000111108C0D095DE23DC938FBFDF91CF916D
:1006B0001F910895DE2BF8CF0F931F93CF93082F30
:1006C000082E000C110B20913C0B022E000C330B5A
:1006D00002171307B9F080933C0BC0E08091430BE5
:1006E000C81780F4EC2FF0E0B8010C2E02C075950D
:1006F00067950A94E2F76170E65CF44F8581AFDF9D
:10070000CF5FECCF8091460B882329F0813041F1F7
:100710008FEF9FEF21C08091450B863308F0865301
:1007200020917B00982F9870277F922B90937B00CD
:100730008770806480937C0080917A0080648093CD
:100740007A0080917A0086FDFCCF909178008091AC
:100750007900892798278927CF911F910F910895B4
:100760008091450BCF911F910F9151CFCF93DF9384
:1007700090E0FC01ED56FE4F2491835B9E4FFC01FF
:1007800084918823C9F090E0880F991FFC01E15003
:10079000FF4FA591B491FC01E75EFE4FC591D49146
:1007A00061110DC09FB7F8948C91209582238C9392
:1007B0008881282328839FBFDF91CF9108956230DD
:1007C00051F49FB7F8943C91822F809583238C93AA
:1007D000E8812E2BEFCF8FB7F894EC912E2B2C9332
:1007E0008FBFEACF3FB7F8948091D3069091D4069B
:1007F000A091D506B091D60626B5A89B05C02F3F7F
:1008000019F00196A11DB11D3FBFBA2FA92F982F36
:100810008827BC01CD01620F711D811D911D42E031
:10082000660F771F881F991F4A95D1F708958F92F9
:100830009F92AF92BF92CF92DF92EF92FF924B01C5
:100840005C01D0DF6B017C01CDDF6C197D098E0965
:100850009F09683E734081059105B0F321E0821A3B
:100860009108A108B10888EEC80E83E0D81EE11CEB
:10087000F11C81149104A104B10431F7FF90EF90B1
:10088000DF90CF90BF90AF909F908F9008952FB73B
:10089000F8946091CF067091D0068091D106909126
:1008A000D2062FBF0895FC01848187FD04C091E02A
:1008B00069276383D4DE80E00895FC01808580FD94
:1008C00004C082FB882780F9089580E00895FC0128
:1008D0009085957081E0953009F080E00895862F2D
:1008E000642F44CFFC01818592DE21E0892B09F43D
:1008F00020E0822F0895DC01ED91FD918081ED9142
:10090000FD919081ED91FD916C9163708E2309F0C2
:1009100064609F2309F06860E8E9F4E0E60FF11DE8
:10092000659565956D936D917D918D919D910994DE
:1009300023C01AC012C016C010C01EC009C014C007
:1009400013C006C019C009C00DC007C00DC014C037
:1009500062507040804090400BC0615070408040B9
:10096000904006C06E5F01C06F5F7F4F8F4F9F4FFB
:100970009E938E937E936E930895CF93DF93EC01B5
:100980008B85823058F4F894CE01B5DF6F8178857D
:1009900089859A857894DF91CF910895F894F6CF60
:1009A00090E0823090F404968330910569F17CF4F4
:1009B00081309105C9F00297F9F0809169008C7F30
:1009C000816080936900E89A08950297EDCF8430A2
:1009D000910511F1059789F780916A00837F846002
:1009E00080936A00ED9A089580916900837F846006
:1009F00080936900E99A0895809169008F7C8061F5
:100A000080936900EA9A0895809169008F738064E9
:100A100080936900EB9A089580916A008C7F8160D1
:100A200080936A00EC9A0895823161F130F482304B
:100A300079F08330A9F080E008958431B9F0E0F0D6
:100A40008531C9F7709361066093600682E005C046
:100A500070935D0660935C0680E0A2DF81E00895FC
:100A600070935F0660935E0681E0F7CF7093630634
:100A70006093620683E0F1CF70936506609364062D
:100A800084E0EBCF709367066093660685E0E5CF60
:100A90000F931F93CF93DF93EC01062F142F62E087
:100AA000802F64DE62E0812F61DE802F90E0FC0108
:100AB000E35BFE4FE491F0E0EE0FFF1FED5CFE4FB5
:100AC000A591B491B983A883FC01ED56FE4F249102
:100AD0002C83812F90E0FC01E35BFE4FE491F0E07A
:100AE000EE0FFF1FED5CFE4F459154915B834A83EF
:100AF000FC01ED56FE4FE491ED831F8218861986A6
:100B00001A868BE39FE10197F1F78C91282391E0FE
:100B100009F490E0DA018C91E82309F092609E8359
:100B2000BE01802F81DF8B87BE01812F7DDF9B85FA
:100B3000890F8B87DF91CF911F910F9108958F922D
:100B40009F92AF92BF920F931F93CF93DF93CDB736
:100B5000DEB7A1970FB6F894DEBF0FBECDBF19A2C6
:100B6000423008F44AE08E010F5D1F4F842E912C15
:100B7000B12CA12CA50194010E94270FE62FB901E9
:100B8000CA01EA303CF5E05DD801EE938D01232BDC
:100B9000242B252B79F790E080E0109761F0FD0180
:100BA00001900020E9F73197AF014A1B5B0BBD01B3
:100BB00083E097E0A2DBA1960FB6F894DEBF0FBEEC
:100BC000CDBFDF91CF911F910F91BF90AF909F90BC
:100BD0008F900895E95CD8CF4AE065E070E080E04E
:100BE00090E0ADCF009761F0FC0101900020E9F7A3
:100BF0003197AF01481B590BBC0183E097E07DCBD7
:100C000090E080E008950F931F93CF93DF9383E0EC
:100C100097E0DADB892B09F44EC083E097E0B2DB82
:100C20008C37C1F48DEE90E052DC8CE393E0DADF98
:100C30008BEE90E04CDCD0DF89EE90E048DC8EE07B
:100C400092E0D0DF87EE90E042DC84DB84EE90E03F
:100C50003EDCDDCF8C3329F41092CD061092CC0609
:100C6000D6CF8A30B1F4CEE1D2E008E616E0899121
:100C70009991009739F0F801208161E0213309F062
:100C800060E0EDDC0F5F1F4FF2E0C632DF0779F75F
:100C9000E3CF2091CC063091CD0624363105E4F621
:100CA000F901E859F94F80832F5F3F4F3093CD060C
:100CB0002093CC06ACCFDF91CF911F910F91089577
:100CC0008FDB8111A0DF80E090E0892B49F080E08C
:100CD00090E0892B29F00E94000081110E94000001
:100CE00080E090E0892B49F080E090E0892B29F0AA
:100CF0000E94000081110E94000080E090E0892B9A
:100D000049F080E090E0892B29F00E9400008111D9
:100D10000C9400000895AF92BF92DF92EF92FF9281
:100D20000F931F93CF93DF93EC01D62EF42E122F47
:100D300084E090E00E946D0FFC01F0821183028339
:100D4000E3828AE193E0998388838FEF8A838B83A0
:100D50008C838A878B878C8784E089878F015E01EB
:100D600085E0A80EB11CF12CF80181918F0187FD5F
:100D700033C0F50181935F0161E0F8DCF394F4E0A6
:100D8000FF12F2CF8FEF8C8380E293E09983888308
:100D90008B8587FD0FC0282F082E000C330BD21631
:100DA000130641F09A85913011F460E058DC60E060
:100DB0008B85DCDC82E08A87DB8662E08D2DD6DCE9
:100DC00081E08C87DF91CF911F910F91FF90EF9081
:100DD000DF90BF90AF900895F986D4CF0E946E1136
:100DE0000F931F93CF93DF93EC0188819981009734
:100DF00059F02A813B812617370730F081E0DF91D7
:100E0000CF911F910F9108958B016F5F7F4F0E94CB
:100E10009210009759F0998388831B830A832C8151
:100E20003D81232B59F7FC011082E8CF80E0E7CF0A
:100E3000CF93DF93EC0188819981009711F00E9494
:100E40000910198218821D821C821B821A82DF916E
:100E5000CF910895EF92FF920F931F93CF93DF935B
:100E6000EC017B018A01BA01BBDF81110AC0CE010E
:100E7000DFDFCE01DF91CF911F910F91FF90EF90B7
:100E800008951D830C83B701888199810E94831185
:100E9000F0CFCF93DF93EC01FB018617970741F06A
:100EA000608171816115710539F044815581D2DF0E
:100EB000CE01DF91CF910895BBDFFACFFC01808195
:100EC0009181009711F00C94091008951F920F92D0
:100ED0000FB60F9211240BB60F922F933F934F939F
:100EE0005F936F937F938F939F93AF93BF93EF9392
:100EF000FF9383E097E07DDAFF91EF91BF91AF918F
:100F00009F918F917F916F915F914F913F912F9121
:100F10000F900BBE0F900FBE0F901F9018951F9251
:100F20000F920FB60F9211240BB60F922F938F933F
:100F30009F93EF93FF93E0911307F0911407808143
:100F4000E0911907F0911A0782FD1DC090818091F0
:100F50001C078F5F8F7320911D07821741F0E0916E
:100F60001C07F0E0ED5FF84F958F80931C07FF9111
:100F7000EF919F918F912F910F900BBE0F900FBE0D
:100F80000F901F9018958081F2CF1F920F920FB68D
:100F90000F9211242F933F938F939F93AF93BF93FF
:100FA0008091CF069091D006A091D106B091D20643
:100FB0003091CE0623E0230F2D3758F50196A11D61
:100FC000B11D2093CE068093CF069093D006A093B8
:100FD000D106B093D2068091D3069091D406A09109
:100FE000D506B091D6060196A11DB11D8093D306FA
:100FF0009093D406A093D506B093D606BF91AF9137
:101000009F918F913F912F910F900FBE0F901F9046
:10101000189526E8230F0296A11DB11DD2CF1F926D
:101020000F920FB60F9211240BB60F922F933F938E
:101030004F935F936F937F938F939F93AF93BF93E0
:10104000EF93FF9380915E0690915F0654DCFF91D1
:10105000EF91BF91AF919F918F917F916F915F9130
:101060004F913F912F910F900BBE0F900FBE0F909D
:101070001F9018951F920F920FB60F9211240BB666
:101080000F922F933F934F935F936F937F938F9321
:101090009F93AF93BF93EF93FF9380915C069091E2
:1010A0005D0629DCFF91EF91BF91AF919F918F91E8
:1010B0007F916F915F914F913F912F910F900BBE58
:1010C0000F900FBE0F901F9018951F920F920FB6A2
:1010D0000F9211240BB60F922F933F934F935F9370
:1010E0006F937F938F939F93AF93BF93EF93FF93F0
:1010F0008091660690916706FEDBFF91EF91BF91AC
:10110000AF919F918F917F916F915F914F913F919F
:101110002F910F900BBE0F900FBE0F901F90189540
:101120001F920F920FB60F9211240BB60F922F93AE
:101130003F934F935F936F937F938F939F93AF935F
:10114000BF93EF93FF938091640690916506D3DB84
:10115000FF91EF91BF91AF919F918F917F916F918F
:101160005F914F913F912F910F900BBE0F900FBE4B
:101170000F901F9018951F920F920FB60F92112487
:101180000BB60F922F933F934F935F936F937F9381
:101190008F939F93AF93BF93EF93FF9380916206DA
:1011A00090916306A8DBFF91EF91BF91AF919F9162
:1011B0008F917F916F915F914F913F912F910F9000
:1011C0000BBE0F900FBE0F901F9018951F920F929D
:1011D0000FB60F9211240BB60F922F933F934F939C
:1011E0005F936F937F938F939F93AF93BF93EF938F
:1011F000FF9380916006909161067DDBFF91EF91F6
:10120000BF91AF919F918F917F916F915F914F911E
:101210003F912F910F900BBE0F900FBE0F901F901C
:101220001895EF920F93109206071092050788EE1B
:1012300093E0A0E0B0E08093070790930807A093A5
:101240000907B0930A0786E293E09093040780931E
:10125000030785EC90E09093100780930F0784ECD0
:1012600090E0909312078093110780EC90E09093A8
:1012700014078093130781EC90E0909316078093F6
:10128000150782EC90E0909318078093170786EC7F
:1012900090E090931A078093190710921C07109200
:1012A0001D0710921E0710921F07A0EAB7E090E0FA
:1012B00080E041E2FC013E9621E030E0863091057D
:1012C00010F430E020E0E20FF31F40935700E49168
:1012D000ED9301968930910569F787E1E82E09E1E0
:1012E0002BE14DE166E18AE39BE015DD97E6E92E0F
:1012F00006E625E644E663E68DE29BE00CDD43E08E
:1013000062E08DEC9AE0C4DB8CE493E09093DA0A1F
:101310008093D90A87E593E09093DC0A8093DB0AF7
:1013200046E065E08DED9AE0B3DB82E693E09093D2
:10133000EA0A8093E90A8DE693E09093EC0A8093A1
:10134000EB0A43E361E28DEE9AE0A2DB88E793E0EB
:101350009093FA0A8093F90A83E893E09093FC0A49
:101360008093FB0A4FE269E28DEF9AE091DB8EE811
:1013700093E090930A0B8093090B8BE993E0909391
:101380000C0B80930B0B48E16FE38DE09BE080DB5F
:1013900088EA93E090931A0B8093190B89EB93E002
:1013A00090931C0B80931B0B4AE161E48DE19BE061
:1013B0006FDB8AEC93E090932A0B8093290B8BEDE3
:1013C00093E090932C0B80932B0BE5EBF7E028E355
:1013D00033E08AE090E0318320831282138214820A
:1013E0001582978386831086118672964AE0ED3CBB
:1013F000F40789F71092B0071092AF071092B20766
:101400001092B1071092B4071092B30750E040E079
:101410006CE074E08FEA97E01DDD1092AA0710924D
:10142000A9071092AC071092AB071092AE0710926A
:10143000AD074DE050E06CEE73E089EA97E00F9164
:10144000EF9008CDCF93DF93CDB7DEB764970FB69B
:10145000F894DEBF0FBECDBF789484B5826084BDA2
:1014600084B5816084BD85B5826085BD85B58160A8
:1014700085BD80916E00816080936E001092810026
:1014800080918100826080938100809181008160E1
:1014900080938100809180008160809380008091A2
:1014A000B10084608093B1008091B000816080932E
:1014B000B0008091910082608093910080919100B2
:1014C0008160809391008091900081608093900072
:1014D0008091A10082608093A1008091A100816031
:1014E0008093A1008091A00081608093A0008091F2
:1014F000210182608093210180912101816080938C
:1015000021018091200181608093200180917A00E7
:10151000846080937A0080917A00826080937A0060
:1015200080917A00816080937A0080917A0080684F
:1015300080937A001092C100E0911307F091140794
:1015400082E08083E0910F07F09110071082E09114
:101550001107F091120780E1808310921B07E09140
:101560001707F091180786E08083E0911507F09146
:101570001607808180618083E0911507F09116073E
:10158000808188608083E0911507F0911607808143
:1015900080688083E0911507F091160780818F7D28
:1015A000808382E390E0A0E0B0E08093070790930F
:1015B0000807A0930907B0930A0768EE73E080E07C
:1015C00090E035D901EAC02E07E0D02E8E010F5FE2
:1015D0001F4FD6018D916D011B861A861D861C86B4
:1015E0001F861E8640E1B80190E008D4F801019002
:1015F0000020E9F73197AF01401B510BB801CE0134
:101600000A9628DC1A8219821C821B821E821D8285
:101610006FEA77E0C8013DDC8E859F85AA84BB8494
:10162000ED80FE80E80EF91EA114B10499F1892B1A
:1016300079F0B701C801D4DB882361F129813A81AF
:101640008D819E81B501820F931F5DD6FE82ED8252
:10165000B8018FEA97E01DDCC80130DCCE010A96A4
:101660002DDCB9EACB16B7E0DB0609F0B2CF00916A
:10167000AF071091B0070115110579F0F8018081CD
:10168000882359F0082E000C990B2CD6D8018D9385
:101690008D01F4CFC801CCDBDBCF88E292E00E9461
:1016A00067028CE393E09EDA86E292E00E94670292
:1016B00093DA84E292E00E9467028EE092E092DA8E
:1016C00082E292E00E9467020E94AA018FE192E00A
:1016D0000E94670217EDE12E16E0F12E10E0812F37
:1016E0000E945C03F70181937F011F5F1031B9F7FE
:1016F00005EB17E0A6E6EA2EA2E0FA2EBAE0AB2E42
:10170000B12CD701DC9011967C91D801ED91FC9120
:101710000280F381E02D42E050E06D2DC801199563
:10172000F801D18610860190F081E02D0190F081C2
:10173000E02DC8011995882339F0D80118968C91AD
:101740001897836018968C93A2D8F80162837383EC
:1017500084839583B782A682F4E0EF0EF11C0E5EBF
:101760001F4F2AE00D3C120761F6E3E0CE2EE7E0C2
:10177000DE2E0BEE16E0FDECEF2EFAE0FF2EC70199
:10178000FCD8D8016D937D938D939D938D01B0E12D
:10179000EB0EF11CC016D10691F76EE1E62E62E069
:1017A000F62E76E2A72E72E0B72E8701F801C190DF
:1017B000D1908F01C114D10441F061E08C2D0E94C1
:1017C000B60361E08C2D0E942F03A016B10671F7BD
:1017D00068EB7BE080E090E02AD8D7018D919D9165
:1017E0007D01009719F060E00E942F030E151F0580
:1017F000A1F75CE3E52E53E0F52E49D84B015C01DF
:101800008091140290911502A0911602B0911702D6
:10181000AC01BD014854544F6F4F7F4F841695065D
:10182000A606B70628F488169906AA06BB0668F528
:101830008FE792E00E9467028CE393E0D3D98DE7B3
:1018400092E00E946702C8D98BE792E00E9467028B
:101850008EE092E0C7D989E792E00E9467020E9479
:10186000AA0186E792E00E94670280921402909299
:101870001502A0921602B092170280920A0290926C
:101880000B02A0920C02B0920D024BEEC42E46E069
:10189000D42E0DEC1AE091E0BAEFEB16B3E0FB06A4
:1018A00009F090E0F80124853585F3E02C343F07FA
:1018B00009F419C12857334009F415C1D8011E96FF
:1018C0002D913C9181E0B3E027353B0721F023586F
:1018D000334009F080E0992309F407C1882309F413
:1018E00004C1C8014AD824E030E040E050E0D1D241
:1018F00029013A01F60180819181A281B381841589
:101900009505A605B7050CF0F8C0D8011E968D9177
:101910009C9168D984E792E00E94670280920A0253
:1019200090920B02A0920C02B0920D02D6014D9241
:101930005D926D927D926D01005F1F4FEDE2FBE0C5
:10194000E017F10709F0A7CF36E6632E32E0732ED9
:1019500005EB17E0D12CC12CD80118968C91189763
:101960008B7F18968C931897ED91FC910190F081E4
:10197000E02DC80119958C8BF801808586958170C2
:101980002C88281609F4C6C00E944704D801129674
:101990006D937D938D939C93159718968C91B2E0DF
:1019A0008B27F8018087C8010E945D04811106C061
:1019B000C8010E946704882309F487C0F30180816D
:1019C00091819C012B7F2332310509F44EC08B326B
:1019D000910509F44AC08D32910509F446C031E001
:1019E000FDE0EF16F4E0FF0609F030E0AC014353F0
:1019F000510921E04230510520F08032910509F073
:101A000020E0332311F0211130C020E2E21624E05F
:101A1000F20609F4CDC046E3E41644E0F40609F406
:101A2000C7C05CE4E51654E0F50609F4C1C021E046
:101A3000A1E6EA16A4E0FA0631F0B7E7EB16B4E047
:101A4000FB0609F020E0AC01435151094330510538
:101A500008F4B0C041E08C31910509F040E0222348
:101A600009F4AAC0442309F4A7C080920602909208
:101A70000702A0920802B09209021092EA061092A0
:101A8000E906D30112968D919C91ACD8C8010E94B1
:101A90005D04882309F493C18EE692E00E946702F8
:101AA0008FE592E0B4E0CB16D10409F499C164E665
:101AB00070E080E090E00E94170480920A02909209
:101AC0000B02A0920C02B0920D02FFEFCF1ADF0AB8
:101AD0000E5E1F4F24E0620E711C3CE2C316D1045F
:101AE00009F03ACFCCC081E0F6CEC8010E94BD0417
:101AF00022E030E040E050E0FACE481659066A068F
:101B00007B060CF013CFF801848595856BD882E7AE
:101B100092E002CF0E944704D80112962D903D908A
:101B20004D905C9015979B01AC0122193309440933
:101B3000550916968D919C91B0E0A0E028173907C1
:101B40004A075B0708F42FCFD80118968C91817053
:101B50002C88281609F427CF0E944704D801129632
:101B60006D937D938D939C93159718968C91B1E00E
:101B70008B278460F80180870E944704D8011A9659
:101B80002D913D914D915C911D97621B730B840BC0
:101B9000950BF80166877787808B918B0E944704AD
:101BA000D8011A966D937D938D939C931D97FBCED0
:101BB00021E049CF41E053CF8532910549F182338D
:101BC000910511F4311124C0E0E2EE16E4E0FE06C6
:101BD00009F4F3C0F6E3EF16F4E0FF0609F4EDC0F4
:101BE0002CE4E21624E0F20609F4E7C021E031E635
:101BF000E31634E0F30631F047E7E41644E0F40678
:101C000009F020E04A9709F03CCF222309F439CFAC
:101C10008091060290910702A0910802B0910902FA
:101C200083589F4FAF4FBF4F88169906AA06BB0631
:101C300030F181E090E09093EA068093E906D0923B
:101C4000E806C092E7068092020290920302A092F8
:101C50000402B0920502C8010E945D04882321F0AD
:101C60001092010210920002C8010E9467048823AA
:101C700031F081E090E0909301028093000261E0F6
:101C800070E080E090E00E94170406E212E027ED89
:101C9000C22E26E0D22E712C872D0E945C03682E66
:101CA000D6018D916D01681699F0FD013197608222
:101CB000F801828193810E94F20588E492E0662017
:101CC00029F0F1E06F1204C084E492E00E94670200
:101CD00073940C5F1F4F90E1292E7210DDCF80911D
:101CE0000A0290910B02A0910C02B0910D02AC017E
:101CF000BD014C595F4F6F4F7F4F84169506A60666
:101D0000B70628F488169906AA06BB0660F482E492
:101D100092E00E94670280920A0290920B02A092C7
:101D20000C02B0920D028091020290910302A091E8
:101D30000402B091050283589F4FAF4FBF4F8815E3
:101D40009905AA05BB05B0F58091E9069091EA06D0
:101D5000019781F5E091E706F091E806EE0FFF1F8D
:101D6000EE0FFF1FEA59FD4F828193810E94F20519
:101D700080910002909101020097A9F58EE392E014
:101D80000E94670264E670E080E090E00E94170421
:101D900080920A0290920B02A0920C02B0920D0265
:101DA0001092EA061092E90689E090E09093010211
:101DB000809300020E94600620CD21E023CFC8015D
:101DC0000E946704882309F472CE8BE592E00E949A
:101DD0006702E4E0CE16D10409F069CE8CE492E00B
:101DE0000E94670264CE019769F68AE392E0C8CF49
:101DF00089EA97E063D88FEA97E060C8BB27FB01C8
:101E00005527AA27880F991FAA1FA41710F0A41BF3
:101E100083955051B9F7A05DAA3308F0A95DA1934D
:101E2000009779F7B111B1931192CB0100C0DC0199
:101E3000FC01672F71917723E1F7329704C07C9101
:101E40006D9370836291AE17BF07C8F30895A1E246
:101E50001A2EAA1BBB1BFD010DC0AA1FBB1FEE1F24
:101E6000FF1FA217B307E407F50720F0A21BB30B6F
:101E7000E40BF50B661F771F881F991F1A9469F7EB
:101E800060957095809590959B01AC01BD01CF0147
:101E90000895052E97FB16F400940FD057FD05D03A
:101EA000D6DF07FC02D046F408C050954095309527
:101EB00021953F4F4F4F5F4F0895909580957095B6
:101EC00061957F4F8F4F9F4F0895EE0FFF1F881F23
:101ED0008BBF0790F691E02D19940F931F93CF932A
:101EE000DF938230910510F482E090E0E091490B9D
:101EF000F0914A0B30E020E0B0E0A0E0309799F498
:101F00002115310509F44AC0281B390B243031054D
:101F1000D8F58A819B816115710589F1FB01938355
:101F20008283FE0111C040815181028113814817D3
:101F30005907E0F04817590799F4109761F0129685
:101F40000C93129713961C933296CF01DF91CF9189
:101F50001F910F9108950093490B10934A0BF4CFF2
:101F60002115310551F04217530738F0A901DB0163
:101F70009A01BD01DF01F801C1CFEF01F9CF9093C4
:101F80004A0B8093490BCDCFFE01E20FF31F8193E3
:101F900091932250310939832883D7CF2091470B61
:101FA0003091480B232B41F420911A0230911B02EF
:101FB0003093480B2093470B20911802309119025F
:101FC0002115310541F42DB73EB740911C025091C7
:101FD0001D02241B350BE091470BF091480BE217D3
:101FE000F307A0F42E1B3F0B2817390778F0AC013C
:101FF0004E5F5F4F2417350748F04E0F5F1F509319
:10200000480B4093470B819391939FCFF0E0E0E022
:102010009CCFCF93DF930097E9F0FC0132971382B6
:102020001282A091490BB0914A0BED0130E020E003
:102030001097A1F420813181820F931F2091470BCB
:102040003091480B2817390709F061C0F093480B0D
:10205000E093470BDF91CF910895EA01CE17DF0798
:10206000E8F54A815B819E0141155105B1F7E9010F
:10207000FB83EA8349915991C40FD51FEC17FD07E3
:1020800061F4808191810296840F951FE901998303
:102090008883828193819B838A83F0E0E0E01296BB
:1020A0008D919C9113970097B9F52D913C911197C3
:1020B000CD010296820F931F2091470B3091480B60
:1020C0002817390739F6309751F510924A0B1092BC
:1020D000490BB093480BA093470BBCCFD383C2836B
:1020E00040815181840F951FC817D90761F44E5F55
:1020F0005F4F88819981480F591F518340838A819E
:102100009B81938382832115310509F0B0CFF09331
:102110004A0BE093490B9ECFFD01DC01C0CF138237
:102120001282D7CF4F925F926F927F928F929F923F
:10213000AF92BF92CF92DF92EF92FF920F931F93D5
:10214000CF93DF938C01009791F4CB01DF91CF9176
:102150001F910F91FF90EF90DF90CF90BF90AF90C5
:102160009F908F907F906F905F904F90B6CEFC01C4
:10217000E60FF71F9C0122503109E217F30708F41C
:10218000AAC0D901CD91DC911197C617D70718F1D4
:10219000C530D10570F0CE0104978617970748F037
:1021A000C61BD70B2297C193D1936D937C93CF011C
:1021B00030DFC801DF91CF911F910F91FF90EF9019
:1021C000DF90CF90BF90AF909F908F907F906F9057
:1021D0005F904F9008955B01AC1ABD0A4C018C0EC4
:1021E0009D1EA091490BB0914A0B512C412CF12C12
:1021F000E12C109731F58091470B9091480B881591
:10220000990509F05CC04616570608F058C0809141
:10221000180290911902009741F48DB79EB7409132
:102220001C0250911D02841B950BE817F90708F05A
:1022300052C0F093480BE093470BF9017183608320
:10224000B8CF8D919C91119712966C90129713961E
:102250007C901397A815B90559F56C0142E0C40E9E
:10226000D11CCA14DB0420F1AC014A195B09DA0164
:102270001296159780F06282738251834083D90150
:102280006D937C93E114F10471F0D7011396FC93E4
:10229000EE9312978ECF22968C0F9D1FF90191839A
:1022A0008083F301EFCFF0934A0BE093490B81CF8A
:1022B0004816590608F42C017D01D3019ACFCB01B1
:1022C0000CDE7C01009739F0AE01B80113D0C801D3
:1022D000A0DE87016ECF10E000E06BCF81E090E0E0
:1022E000F89418C09111089581568A5108F48052CB
:1022F00085580895FB01DC0102C001900D92415008
:102300005040D8F70895FB01DC0101900D920020A8
:10231000E1F7089511E0CAE4D1E000E005C0802FA4
:10232000FE01D3DD2196011DCB34D10780E00807E3
:06233000B1F7F894FFCFA5
:102336000900FFFFFFFFFFFFFFFFFFFFFFFF332E39
:10234600322E3400FFFFFFFF00004B0B80000F0012
:1023560011001300150000008D0401009304020013
:10236600990403009F040400A5040500AB040600BD
:10237600B1040700B7040800BD040900C3040A003D
:10238600C9040B00CF040C00D5040D00DB040E00BD
:10239600E1040F00E7043500ED040400FA04070029
:1023A60007050800140509001C050A0027050B008F
:1023B6002F050C0037050D0040050E0049051000DD
:1023C600520512005A05140062051E006B051F0017
:1023D60071052000790522007F052300850524006C
:1023E6009005250096052600A3052700A9052800C7
:1023F600B6052A00BC052B00C2052C00CD052D0014
:10240600D3052E00E1053000E9053200EF05340062
:10241600F5053600FE053700040638000A063900C1
:1024260010063A0016063B001C063C0022063E003B
:1024360028064000320642003F0643004506440097
:102446004B064500510600000000EE0600000000A5
:102456005304000000001B027D01B3018102E40168
:10246600C201D6010000000072046F045265616C5F
:1024760053696D476561722D47435500454E435F6D
:102486004844475F555000454E435F4844475F44C4
:102496004E00454E435F4352535F555000454E43F1
:1024A6005F4352535F444E00454E435F414C545F79
:1024B600555000454E435F414C545F444E00454ED7
:1024C600435F52414E47455F444E00454E435F527F
:1024D600414E47455F555000454E435F464D535F5D
:1024E600494E4E45525F555000454E435F464D534B
:1024F6005F494E4E45525F444E00454E435F464D42
:10250600535F4F555445525F555000454E435F4605
:102516004D535F4F555445525F444E00373536454F
:10252600364237373639393939005265616C536965
:102536006D476561722D47464335303000526561FF
:102546006C53696D476561722D47435534373900C1
:102556005265616C53696D476561722D4731303044
:102566003050464431005265616C53696D47656170
:10257600722D47313030304D464431005265616C22
:1025860053696D476561722D473130303058464486
:10259600005265616C53696D476561722D47313034
:1025A600303058464431005265616C53696D476559
:1025B60061722D4731303030584644320042544E15
:1025C6005F5A0042544E5F430042544E5F490042F8
:1025D600544E5F4E0042544E5F540042544E5F5973
:1025E6000042544E5F420042544E5F480042544EF1
:1025F6005F4D0042544E5F530042544E5F580042B6
:10260600544E5F410042544E5F470042544E5F4C69
:102616000042544E5F520042544E5F570042544EA1
:102626005F414C545F53594E430042544E5F4844F9
:10263600475F53594E430042544E5F4352535F53D4
:10264600594E430042544E5F454E540042544E5F2D
:102656004449524543540042544E5F46504C004252
:10266600544E5F434C520042544E5F4D454E55000A
:1026760042544E5F50524F430042544E5F464C49BF
:10268600500042544E5F464D530042544E5F434FF6
:102696004D0042544E5F585044520042544E5F44DF
:1026A6000042544E5F4E41560042544E5F4A00422D
:1026B600544E5F4F0042544E5F50414E5F5550009E
:1026C60042544E5F550042544E5F50414E5F53593F
:1026D6004E430042544E5F450042544E5F50414EB9
:1026E6005F4C4546540042544E5F4B0042544E5F89
:1026F600500042544E5F50414E5F444E0042544E8D
:102706005F560042544E5F50414E5F52494748540F
:102716000042544E5F5350430042544E5F460042BF
:10272600544E5F510042544E5F424B535000425448
:102736004E5F320042544E5F350042544E5F3800C1
:1027460042544E5F300042544E5F330042544E5F57
:10275600360042544E5F390042544E5F4D494E5545
:10276600530042544E5F464D535F53594E43004209
:10277600544E5F310042544E5F340042544E5F3730
:0C2786000042544E5F504552494F440041
:00000001FF
